BL51 BANKED LINKER/LOCATER V6.22                                                        02/06/2018  17:04:01  PAGE 1


BL51 BANKED LINKER/LOCATER V6.22, INVOKED BY:
C:\KEIL\C51\BIN\BL51.EXE main.obj, Delay_1T.obj TO MA82G5Dxx RAMSIZE (256)


MEMORY MODEL: SMALL


INPUT MODULES INCLUDED:
  main.obj (MAIN)
  Delay_1T.obj (DELAY_1T)
  C:\KEIL\C51\LIB\C51S.LIB (?C_STARTUP)


LINK MAP OF MODULE:  MA82G5Dxx (MAIN)


            TYPE    BASE      LENGTH    RELOCATION   SEGMENT NAME
            -----------------------------------------------------

            * * * * * * *   D A T A   M E M O R Y   * * * * * * *
            REG     0000H     0008H     ABSOLUTE     "REG BANK 0"
            DATA    0008H     0002H     UNIT         ?DT?MAIN
            IDATA   000AH     0001H     UNIT         ?STACK

            * * * * * * *   C O D E   M E M O R Y   * * * * * * *
            CODE    0000H     0003H     ABSOLUTE     
            CODE    0003H     00DFH     UNIT         ?PR?_I2C_READ?MAIN
            CODE    00E2H     00A9H     UNIT         CODE_DELAY
            CODE    018BH     0099H     UNIT         ?PR?_I2C_WRITE?MAIN
            CODE    0224H     003CH     UNIT         ?PR?MAIN?MAIN
            CODE    0260H     001CH     UNIT         ?PR?TWI0_INIT?MAIN
            CODE    027CH     000FH     UNIT         ?PR?TIMER0_INITIAL?MAIN
            CODE    028BH     000CH     UNIT         ?C_C51STARTUP



OVERLAY MAP OF MODULE:   MA82G5Dxx (MAIN)


SEGMENT
  +--> CALLED SEGMENT
---------------------
?C_C51STARTUP
  +--> ?PR?MAIN?MAIN

?PR?MAIN?MAIN
  +--> ?PR?TIMER0_INITIAL?MAIN
  +--> ?PR?TWI0_INIT?MAIN
  +--> ?PR?_I2C_WRITE?MAIN
  +--> ?PR?_I2C_READ?MAIN



SYMBOL TABLE OF MODULE:  MA82G5Dxx (MAIN)

  VALUE           TYPE          NAME
  ----------------------------------

BL51 BANKED LINKER/LOCATER V6.22                                                      02/06/2018  17:04:01  PAGE 2


  -------         MODULE        MAIN
  C:0000H         SYMBOL        _ICE_DUMMY_
  D:0095H         PUBLIC        P2M0
  D:0092H         PUBLIC        P2M1
  D:0090H         PUBLIC        P1
  D:00A0H         PUBLIC        P2
  D:00C0H         PUBLIC        XICON
  D:00B0H         PUBLIC        P3
  D:00E8H         PUBLIC        P4
  D:00F8H         PUBLIC        P6
  D:00ACH         PUBLIC        SFRPI
  D:00A8H         PUBLIC        IE
  D:00B8H         PUBLIC        IP0L
  C:0260H         PUBLIC        TWI0_Init
  C:0003H         PUBLIC        _I2C_Read
  D:00D8H         PUBLIC        CCON
  C:0224H         PUBLIC        main
  C:018BH         PUBLIC        _I2C_Write
  D:0008H         PUBLIC        TWI0_Err
  D:0089H         PUBLIC        TMOD
  D:0088H         PUBLIC        TCON
  D:008CH         PUBLIC        TH0
  D:008AH         PUBLIC        TL0
  D:0009H         PUBLIC        tmp
  B:0088H.4       PUBLIC        TR0
  C:027CH         PUBLIC        Timer0_Initial
  D:0098H         PUBLIC        S0CON
  D:00C8H         PUBLIC        T2CON
  D:00A3H         PUBLIC        AUXR2
  D:00A4H         PUBLIC        AUXR3
  D:00D2H         PUBLIC        SIDAT
  D:00D0H         PUBLIC        PSW
  D:00D4H         PUBLIC        SICON
  -------         PROC          _I2C_READ
  D:0007H         SYMBOL        Dev_Addr
  D:0005H         SYMBOL        Reg_Addr
  -------         DO            
  D:0006H         SYMBOL        usData
  D:0002H         SYMBOL        cnt
  C:00DEH         SYMBOL        TWI0R_End
  -------         ENDDO         
  C:0003H         LINE#         30
  C:0003H         LINE#         31
  C:0003H         LINE#         32
  C:0005H         LINE#         33
  C:0007H         LINE#         35
  C:000AH         LINE#         36
  C:000DH         LINE#         37
  C:000DH         LINE#         38
  C:0012H         LINE#         39
  C:0012H         LINE#         40
  C:0017H         LINE#         41
  C:0020H         LINE#         42
  C:0020H         LINE#         43
  C:0020H         LINE#         44
  C:0023H         LINE#         45
  C:0023H         LINE#         46
BL51 BANKED LINKER/LOCATER V6.22                                                      02/06/2018  17:04:01  PAGE 3


  C:0023H         LINE#         47
  C:0026H         LINE#         49
  C:0028H         LINE#         50
  C:002BH         LINE#         51
  C:002EH         LINE#         52
  C:0033H         LINE#         53
  C:0033H         LINE#         54
  C:0038H         LINE#         55
  C:0041H         LINE#         56
  C:0041H         LINE#         57
  C:0041H         LINE#         58
  C:0044H         LINE#         59
  C:0044H         LINE#         60
  C:0044H         LINE#         62
  C:0046H         LINE#         63
  C:0049H         LINE#         64
  C:004CH         LINE#         65
  C:0051H         LINE#         66
  C:0051H         LINE#         67
  C:0056H         LINE#         68
  C:005FH         LINE#         69
  C:005FH         LINE#         70
  C:005FH         LINE#         71
  C:0061H         LINE#         72
  C:0061H         LINE#         73
  C:0061H         LINE#         76
  C:0064H         LINE#         77
  C:0067H         LINE#         78
  C:006AH         LINE#         79
  C:006FH         LINE#         80
  C:006FH         LINE#         81
  C:0074H         LINE#         82
  C:007DH         LINE#         83
  C:007DH         LINE#         84
  C:007DH         LINE#         85
  C:007FH         LINE#         86
  C:007FH         LINE#         87
  C:007FH         LINE#         88
  C:0082H         LINE#         90
  C:0087H         LINE#         91
  C:008AH         LINE#         92
  C:008DH         LINE#         93
  C:0092H         LINE#         94
  C:0092H         LINE#         95
  C:0097H         LINE#         96
  C:00A0H         LINE#         97
  C:00A0H         LINE#         98
  C:00A0H         LINE#         99
  C:00A2H         LINE#         100
  C:00A2H         LINE#         101
  C:00A2H         LINE#         103
  C:00A5H         LINE#         104
  C:00A8H         LINE#         105
  C:00ADH         LINE#         106
  C:00ADH         LINE#         107
  C:00B2H         LINE#         108
  C:00BBH         LINE#         109
BL51 BANKED LINKER/LOCATER V6.22                                                      02/06/2018  17:04:01  PAGE 4


  C:00BBH         LINE#         110
  C:00BBH         LINE#         111
  C:00BDH         LINE#         112
  C:00BDH         LINE#         113
  C:00BDH         LINE#         114
  C:00BFH         LINE#         116
  C:00C2H         LINE#         117
  C:00C5H         LINE#         118
  C:00C8H         LINE#         119
  C:00CDH         LINE#         120
  C:00CDH         LINE#         121
  C:00D2H         LINE#         122
  C:00DBH         LINE#         123
  C:00DBH         LINE#         124
  C:00DEH         LINE#         125
  C:00DEH         LINE#         126
  C:00DEH         LINE#         127
  C:00DEH         LINE#         128
  C:00DEH         LINE#         129
  C:00E1H         LINE#         130
  -------         ENDPROC       _I2C_READ
  -------         PROC          _I2C_WRITE
  D:0007H         SYMBOL        Dev_Addr
  D:0005H         SYMBOL        Reg_Addr
  D:0003H         SYMBOL        ucData
  -------         DO            
  D:0082H         SYMBOL        cnt
  C:0222H         SYMBOL        TWI0W_End
  -------         ENDDO         
  C:018BH         LINE#         132
  C:018BH         LINE#         133
  C:018BH         LINE#         134
  C:018BH         LINE#         135
  C:018EH         LINE#         136
  C:0191H         LINE#         137
  C:0196H         LINE#         138
  C:019BH         LINE#         139
  C:019BH         LINE#         140
  C:019CH         LINE#         141
  C:01A7H         LINE#         142
  C:01A7H         LINE#         143
  C:01A7H         LINE#         144
  C:01A9H         LINE#         145
  C:01A9H         LINE#         146
  C:01A9H         LINE#         147
  C:01ACH         LINE#         149
  C:01AEH         LINE#         150
  C:01B1H         LINE#         151
  C:01B6H         LINE#         152
  C:01BBH         LINE#         153
  C:01BBH         LINE#         154
  C:01BCH         LINE#         155
  C:01C7H         LINE#         156
  C:01C7H         LINE#         157
  C:01C7H         LINE#         158
  C:01C9H         LINE#         159
  C:01C9H         LINE#         160
BL51 BANKED LINKER/LOCATER V6.22                                                      02/06/2018  17:04:01  PAGE 5


  C:01C9H         LINE#         162
  C:01CBH         LINE#         163
  C:01CEH         LINE#         164
  C:01D3H         LINE#         165
  C:01D8H         LINE#         166
  C:01D8H         LINE#         167
  C:01D9H         LINE#         168
  C:01E4H         LINE#         169
  C:01E4H         LINE#         170
  C:01E4H         LINE#         171
  C:01E6H         LINE#         172
  C:01E6H         LINE#         173
  C:01E6H         LINE#         175
  C:01E8H         LINE#         176
  C:01EBH         LINE#         177
  C:01F0H         LINE#         178
  C:01F5H         LINE#         179
  C:01F5H         LINE#         180
  C:01F6H         LINE#         181
  C:0201H         LINE#         182
  C:0201H         LINE#         183
  C:0201H         LINE#         184
  C:0203H         LINE#         185
  C:0203H         LINE#         186
  C:0203H         LINE#         188
  C:0206H         LINE#         189
  C:0209H         LINE#         190
  C:020EH         LINE#         191
  C:0213H         LINE#         192
  C:0213H         LINE#         193
  C:0214H         LINE#         194
  C:021FH         LINE#         195
  C:021FH         LINE#         196
  C:0222H         LINE#         197
  C:0222H         LINE#         198
  C:0222H         LINE#         199
  C:0222H         LINE#         200
  C:0222H         LINE#         201
  C:0223H         LINE#         202
  -------         ENDPROC       _I2C_WRITE
  -------         PROC          TIMER0_INITIAL
  C:027CH         LINE#         204
  C:027CH         LINE#         205
  C:027CH         LINE#         206
  C:027FH         LINE#         207
  C:0282H         LINE#         208
  C:0285H         LINE#         209
  C:0287H         LINE#         210
  C:028AH         LINE#         212
  -------         ENDPROC       TIMER0_INITIAL
  -------         PROC          TWI0_INIT
  C:0260H         LINE#         214
  C:0260H         LINE#         215
  C:0260H         LINE#         216
  C:0263H         LINE#         218
  C:0266H         LINE#         219
  C:0269H         LINE#         220
BL51 BANKED LINKER/LOCATER V6.22                                                      02/06/2018  17:04:01  PAGE 6


  C:026FH         LINE#         221
  C:0272H         LINE#         222
  C:0273H         LINE#         223
  C:0274H         LINE#         224
  C:0275H         LINE#         225
  C:0278H         LINE#         226
  C:027BH         LINE#         227
  -------         ENDPROC       TWI0_INIT
  -------         PROC          MAIN
  C:0224H         LINE#         229
  C:0224H         LINE#         230
  C:0224H         LINE#         231
  C:0227H         LINE#         232
  C:022AH         LINE#         235
  C:022AH         LINE#         236
  C:022AH         LINE#         237
  C:022DH         LINE#         238
  C:0236H         LINE#         239
  C:023AH         LINE#         240
  C:023AH         LINE#         241
  C:023DH         LINE#         242
  C:023DH         LINE#         243
  C:0244H         LINE#         245
  C:0247H         LINE#         246
  C:0250H         LINE#         247
  C:0254H         LINE#         248
  C:0254H         LINE#         249
  C:0257H         LINE#         250
  C:0257H         LINE#         251
  C:025EH         LINE#         253
  -------         ENDPROC       MAIN
  -------         ENDMOD        MAIN

  -------         MODULE        DELAY_1T
  C:00E2H         SEGMENT       CODE_DELAY
  C:0163H         PUBLIC        DELAY_100US
  C:0142H         PUBLIC        DELAY_10US
  C:0125H         PUBLIC        DELAY_1US
  C:016EH         PUBLIC        DELAY_200US
  C:014DH         PUBLIC        DELAY_20US
  C:0128H         PUBLIC        DELAY_2US
  C:0181H         PUBLIC        DELAY_500US
  C:0158H         PUBLIC        DELAY_50US
  C:0137H         PUBLIC        DELAY_5US
  C:00E2H         PUBLIC        _DELAY_MS
  D:00E0H         SYMBOL        ACC
  C:010DH         SYMBOL        DELAY_UNIT_1MS
  N:0001H         SYMBOL        FOSC_12MHZ
  N:0000H         SYMBOL        FOSC_24MHZ
  C:00F0H         SYMBOL        LSB_LOOP
  C:00FDH         SYMBOL        MSB_LOOP0
  C:00FAH         SYMBOL        MSB_LOOP1
  C:00F6H         SYMBOL        NDLSB
  C:0106H         SYMBOL        NDMSB
  C:00E2H         LINE#         29
  C:00E4H         LINE#         30
  C:00E6H         LINE#         31
BL51 BANKED LINKER/LOCATER V6.22                                                      02/06/2018  17:04:01  PAGE 7


  C:00E8H         LINE#         33
  C:00EAH         LINE#         34
  C:00ECH         LINE#         36
  C:00EEH         LINE#         37
  C:00F0H         LINE#         39
  C:00F3H         LINE#         40
  C:00F6H         LINE#         42
  C:00F8H         LINE#         43
  C:00FAH         LINE#         45
  C:00FDH         LINE#         47
  C:0100H         LINE#         48
  C:0103H         LINE#         49
  C:0106H         LINE#         51
  C:0108H         LINE#         52
  C:010AH         LINE#         53
  C:010CH         LINE#         54
  C:010DH         LINE#         57
  C:0110H         LINE#         58
  C:0113H         LINE#         59
  C:0116H         LINE#         60
  C:0119H         LINE#         61
  C:011CH         LINE#         62
  C:011FH         LINE#         63
  C:0122H         LINE#         64
  C:0123H         LINE#         65
  C:0124H         LINE#         66
  C:0125H         LINE#         78
  C:0126H         LINE#         78
  C:0127H         LINE#         79
  C:0128H         LINE#         91
  C:0129H         LINE#         91
  C:012AH         LINE#         91
  C:012BH         LINE#         91
  C:012CH         LINE#         91
  C:012DH         LINE#         91
  C:012EH         LINE#         91
  C:012FH         LINE#         91
  C:0130H         LINE#         91
  C:0131H         LINE#         91
  C:0132H         LINE#         91
  C:0133H         LINE#         91
  C:0134H         LINE#         91
  C:0135H         LINE#         91
  C:0136H         LINE#         92
  C:0137H         LINE#         108
  C:0139H         LINE#         109
  C:013CH         LINE#         110
  C:013FH         LINE#         111
  C:0141H         LINE#         112
  C:0142H         LINE#         127
  C:0144H         LINE#         128
  C:0147H         LINE#         129
  C:014AH         LINE#         130
  C:014CH         LINE#         131
  C:014DH         LINE#         146
  C:014FH         LINE#         147
  C:0152H         LINE#         148
BL51 BANKED LINKER/LOCATER V6.22                                                      02/06/2018  17:04:01  PAGE 8


  C:0155H         LINE#         149
  C:0157H         LINE#         150
  C:0158H         LINE#         165
  C:015AH         LINE#         166
  C:015DH         LINE#         167
  C:0160H         LINE#         168
  C:0162H         LINE#         169
  C:0163H         LINE#         184
  C:0165H         LINE#         185
  C:0168H         LINE#         186
  C:016BH         LINE#         187
  C:016DH         LINE#         188
  C:016EH         LINE#         206
  C:0170H         LINE#         207
  C:0173H         LINE#         208
  C:0176H         LINE#         209
  C:0179H         LINE#         210
  C:017CH         LINE#         211
  C:017EH         LINE#         212
  C:017FH         LINE#         212
  C:0180H         LINE#         213
  C:0181H         LINE#         234
  C:0184H         LINE#         235
  C:0187H         LINE#         236
  C:018AH         LINE#         237
  -------         ENDMOD        DELAY_1T

Program Size: data=11.0 xdata=0 code=663
LINK/LOCATE RUN COMPLETE.  0 WARNING(S),  0 ERROR(S)
